:100000000AC018951895189518951FC01895189539
:100010001895189518958FED8DBFC0ECE8EB4E2E16
:10002000DD275D2EEEE7F0E0A0E6B0E088278D93B7
:100030003197E9F7662480E08FBD84E08EBD8E9A0B
:1000400089B7806889BF7894FFCF0F921F922F9253
:100050003F924F925F927F92AF92BF920F931F9306
:100060002F933F934F935F936F937F938F939F93C0
:10007000AF93BF93CF93DF93EF93FF938FB78F939C
:100080008EEE95E89DBD8CBD82B390E4892782BB3E
:100090008F918FBFFF91EF91DF91CF91BF91AF9182
:1000A0009F918F917F916F915F914F913F912F9190
:1000B0001F910F91BF90AF907F905F904F903F90B6
:1000C0002F901F900F9018953197F1F7089568942D
:0A00D00062F80895E89462F80895BC
:00000001FF
